:020000040000FA
:0400000057EF00F0C6
:06002A00D9CFE5FFE1CF94
:10003000D9FF00C0E5FF01C0E5FF02C0E5FF03C036
:10004000E5FF020EDBCF00F0030EDBCF01F000C0B6
:1000500002F001C003F0FF0E0026D8A001060250F6
:10006000031006E0FA0E026E0000022EFDD7EFD755
:10007000E4CF03F0E4CF02F0E4CF01F0E4CF00F0EE
:10008000E4CFD9FF1200620ED36E926A816A006AD1
:10009000100E005CFCE200C080FFE56AC80EE56E51
:1000A00015EC00F0020EE126002AF2D7120012EE43
:1000B000FFF022EEFFF0F86AA68EA69C43EC00F05B
:0200C000FFD768
:00000001FF
